:020000040000FA
:100000008501860107309F0001308A000030A5007D
:10001000831603139F0186008500831203133A2081
:10002000152022202E206B20102830308400103024
:10003000A400240825076E208000840AA40B192838
:10004000A50A0800803043200830A3003F30840018
:1000500000084F208403A30B28280800C030432049
:100060000830A3003730840000084F208403A30B1E
:100070003428080038304320013043200330432027
:100080000F304320080086005B20043085005B2091
:10009000003085005B20043085005B20080086006E
:1000A0005B20063085005B20023085005B20063037
:1000B00085005B2008000A30A200A100A10B5E2889
:1000C000A20B5D280800FA30A200A100A10B66284F
:0E00D000A20B65280800632063200800820050
:100200002034453444345534503449344334203454
:100210003134363446343634323438342E342E3495
:1002200032344B3420344D3445344D344F34523411
:1002300049344134203446344C3441345334483406
:100240002E342E343234323434342034423459345F
:1002500054344534533420344434453420345234F7
:1002600041344D342E342E34313432343834203449
:1002700042345934543445345334203444344534AE
:10028000203445344534503452344F344D342E34B8
:100290002E34503455344534523454344F3453345E
:1002A0002034503441345234413420344C344334BB
:1002B00044342034593420345434453443344C3499
:1002C000413444344F342E342E34523445344C347B
:1002D00045345634413444344F3452342034443459
:1002E0004534203431343234373476342E342034AB
:1002F0003134203461346D3470342E342E3438343B
:1003000020344C344534443453342E342E34343475
:1003100020344D344934433452344F3453345734F9
:100320004934543443344834453453342E342E3411
:10033000503452344F344734523441344D344134C4
:1003400044344F3452342034443445344C34203413
:100350003134363446343634323438342034493447
:100360004E345434453447345234413444344F3499
:100370002E342E3449344E3443344C3455345934AD
:100380004534203453344F34463454345734413494
:100390005234453420344D3450344C34413442349A
:1003A000203443344F344E34203445344E345334A7
:1003B00041344D3442344C34413444344F3452345B
:1003C0002C342034533449344D3455344C34413476
:1003D00044344F34523420345934203443344F346D
:1003E0004D34503449344C34413444344F34523415
:1003F0002E342E342E342E342E342E342E342E34ED
:020400002E3498
:02400E00293F48
:00000001FF
